:030000000219FDE5
:03000B000200AA46
:03002B0002015778
:03005B000202E9B5
:030073000202D6B0
:1000800002030406080C10182030406080040608A3
:100090000C10182030406080A0C00003070F1F0D17
:1000A0000D0403060D0502030202C2AFC0D0C0E07A
:1000B000206214E5256009E473E525F4F58AD2622F
:1000C000D0E0D0D0D2AF3285268AC262E526F46075
:1000D0002AD0E0D0D0C295C294C293D2AF32C2959A
:1000E000C294C293206F0D20650A7405D5E0FDE52A
:1000F0007BF45290D0E0D0D0D2AF32758A00C28D5E
:10010000D26201F401B9306805206502D29501B9C7
:10011000306805206502D29401B930680520650277
:10012000D29301B9D29230680A2065077403D5E0F2
:10013000FDD29501B9D29130680A2065077403D5C4
:10014000E0FDD29401B9D29030680A2065077403AB
:10015000D5E0FDD29301B9C2AFC2AD53E6EFC0D036
:10016000C0E0D2D3D2AFC2CEE52A600720744F15CB
:100170002A21BE7800790020742EE580307E01F4BB
:1001800030E70278FF53DACF207E0343DA20307E57
:100190000343DA10C2D8C271E580307E01F430E743
:1001A0000279FFC3E89970CB306103752A4020744F
:1001B00003752A40885CD270E86003755F00207484
:1001C0000DE52B6004152B21CE43DA01C2D8207037
:1001D0000221E1A85C206102C27020740221DF8844
:1001E000227882B6040385222420CF0AD0E0D0D022
:1001F00043E610D2AD32C2CF053A7802E52A600557
:10020000307402152AC3E55C94014005755F004116
:1002100022756000756900E55F2401F55F50037584
:100220005FFF7982B7020D306E1DC3E52294324024
:1002300016854C227982B7030E306E0BC3E52294EB
:10024000324004798E8722C3E5239522600840045A
:10025000152341560523D8CA0569E5697002156959
:10026000D56A69756A017808E56B60497805C3E568
:1002700069956B4057C3E569956C50087801756ABC
:1002800003020290C3E569956D50057801756A0116
:10029000C3E5629524401E7982B7040241C1206EF5
:1002A00014852462E569046003856B69756A0175CC
:1002B000233C0202CCE5622850057562FF41C1F57E
:1002C00062E5620470067560FF7569FFD0E0D0D00A
:1002D00043E610D2AD32C2AF53E67F7592FA759302
:1002E000FFC260759104D2AF32C2AF53E6EFC2AD28
:1002F000C0D0C0E0C0F0D2D3D2AFA8FBA9FCC2D816
:10030000307102615053DACF207E0343DA10307E21
:100310000343DA20D271E580307E01F420E70261E8
:100320002788278928A13553DACF207E0343DA2096
:10033000307E0343DA10C2D8C271307402A1217832
:1003400000E580307E01F430E702A121885CA1093C
:1003500053DACF207E0343DA20307E0343DA10C223
:1003600071206102812953DACF207E0343DA1030F5
:100370007E0343DA20C2D8D27188578958C3E895E2
:1003800055F8E99556F97B007E087A00C3E8948C0D
:10039000E994005005755B00811B882178A2E6A8CE
:1003A000216055C3E894C8E994005008E4D2E4FB06
:1003B0007A0A61F6C3E89468E994015008E4D2E34C
:1003C000FB7A0F61F6C3E894D0E994025008E4D2B6
:1003D000E2FB7A1E61F6C3E894A0E994055008E4B4
:1003E000D2E1FB7A3C61F6C3E89498E9940850089E
:1003F000E4D2E0FB7A787E00C3E89559FCE9955A8F
:10040000FD30E70AECF42401FCEDF43400FD755BEB
:1004100000C3EC9AED9E5003755B018859895A859B
:1004200057558558567802A109C3E89527F8E995EC
:1004300028F9307C0281ED307B0281ED307A028137
:10044000E6207502814CE9FDE8FC816BE9C313F9F4
:10045000E813F830790281E6E9C313F9E813F830BC
:10046000780281E6E9C313FDE813FC20612CC3EC9C
:0E047000941CED940240028182ED701EC3ECDC
:10047E0094C850180529E52970021529C3E5299459
:10048E000A5002A121755C00D270A121E5296002FB
:10049E0015297400207F037896E624FAFEE43400D2
:1004AE00FFC3EC9EFCED9FFD50067800790081EDB8
:1004BE00C3EC94FFED9400400678FF790081EDECDB
:1004CE008572F0A4C5F0A2F733F879004003020557
:1004DE000978FF7900020509E9C313F9E813F8302A
:1004EE007C0EE9600278FFC3E81338F8E43400F9B3
:1004FE00C3E894FFE99400400278FF885CD2702034
:10050E006102A121741FF4552F4BF52FC274EB70AD
:10051E0002D274752A40307403752A0A306102A122
:10052E003520740353DAFE207403752B20D0F0D0DF
:10053E00E0D0D0D2AD43E6103279010205657903E1
:10054E00020565790A020565791E02056579640260
:10055E00056579C80205657817E4D5E0FDD8FAD9A6
:10056E00F6227A147B7802058C7A107B8C02058C2D
:10057E007A0D7BB402058C7A0B7BC802058CE57371
:10058E00D5E001227902E4D291D5E0FDD294D5E0F6
:10059E00FDC294D5E0FDC291D5E0FDE920E002D286
:1005AE009530E002D293E573D5E0FDE920E002C27A
:1005BE009530E002C2937496D5E0FDD9C9EAF8D51C
:1005CE00E0FDD8FBDBB8D29122C37C007D0075F034
:1005DE000005F0EA33FAEB33FB50F6EB13FBEA13AC
:1005EE00FAC3E9FFE8FEE89AF8E99BF95004EFF93F
:1005FE00EEF8B3EC33FCED33FDD5F0DFEDF9ECF8AE
:10060E0022E889F08A20D2D4F8A9F07B0030F70BCB
:10061E007BFFF42401F8E9F43400F9E88520F0A416
:10062E00ADF0F8E98520F0A4AFF0FEED2EF97400E0
:10063E003FFA7C04C3EA13FAE913F9E813F8DCF481
:10064E008BF030F70AE8F42401F8E9F43400F9E805
:10065E0089F0C2D4F8A9F0227882B6040302070505
:10066E00C3E55C9419401EE52D54067018206E36B5
:10067E0078057994E7146007780A1460027812C33B
:10068E00E54198401F306E098564627569FF756A91
:10069E0001852224E4F544F545F546F547F548C2B3
:1006AE006E020705D26E7994E7147013E523F433C6
:1006BE0033F913F8E9540104F9E854FE0206F9E798
:1006CE0014147014E523F4333333F913F8E9540397
:1006DE0004F9E854FC020701E523F433333333F90C
:1006EE0013F8E954070404F9E854F8C39440F8E900
:1006FE009400F98844894522C3E54113F9E5401376
:10070E00F8C3E54498F8E54599F9500CC3E8948090
:10071E00E994FF401602073DC3E8947FE994005028
:10072E000302073D787F790002073D788079FF88C4
:10073E0049894A22E5492546F8E54A3547F9854A69
:10074E0020E4300701F43548FA30E709C3EA94F0A3
:10075E00401502077BC3EA940F500302077B78FF14
:10076E0079FF7A0F02077B780079007AF0C3E524CF
:10077E009561500AC374019524500B020799E54AFE
:10078E0020E70E020799E54A30E706884689478A30
:10079E00482278A5E6FAC3E54933F8E54A33F9D19C
:1007AE000FE930E70BC3E89480E994FF4013E1D3DF
:1007BE00C3E8947FE994005002E1D3787F7900E199
:1007CE00D3788079FFE820E715C3E52398F8400930
:1007DE00C3E8940140030207FA78010207FAE8F42D
:1007EE0024012523F840030207FA78FF884B22786C
:1007FE00A6E6FAA847A94812060FE930E70CC3E8A7
:10080E009401E994FF401602082FC3E894FFE9947F
:10081E0000500302082F78FF790002082F78017923
:10082E00FFE920E715C3E54B98F84009C3E89401AA
:10083E0040030208567801020856E8F42401254BBD
:10084E00F8400302085678FF88242278FF20692892
:10085E0079A1E76023E541601F74FF8541F084852F
:0E086E0039F0306A0375F005A4F8C5F0600299
:10087C0078FFC3E895645002A864886322C3E540FE
:10088C009440E5419401E563500314019A0460021D
:10089C00F563227883E6F520120F1C75E89012059B
:1008AC004775E89030EDFDA8BDA9BE120FC3756E5B
:1008BC0055756F00C3740013FD7455606613FC749A
:1008CC00552CFC74003DFDECFAEDFBC3E89AE99B5A
:1008DC004014E56E2455F56EE56F3400F56FEA2C87
:1008EC00FAEB3DFB80E5AE6EAF6FC3E56F13F9E538
:1008FC006E13F8C3E913F9E813F87A03C3E913F993
:10090C00E813F8DAF7AA201A7009756E00756F00F3
:10091C0002092F1AEA6008EE28FEEF39FFDAF88E8A
:10092C006E8F6F2275E890227883E6FF30EDF9A880
:10093C00BDA9BE0570C3E57094084052757000E9FE
:10094C00FA79A0E76044EA7007E571601B02096858
:10095C00C3E895716010E5715006600C14020974BF
:10096C000460F9020974E571F571C3946D401B754F
:10097C0061C0C394044013756180C39404400B752B
:10098C006140C39404400375610075BB0622EFC33C
:10099C009401601F7455601BC3E894FFE9940350E5
:1009AC0012C3E8956EE9956F5009E561600C15610D
:1009BC000209C6E561F460020561A861C3E52498EB
:1009CC005002A824C3E89562400AA862E562F4606C
:1009DC000385626188258826E570B4070375BB1012
:1009EC0022743279A787F0A4C5F0A2F733F8C3E8D4
:1009FC0095614002A861882288248825882688640D
:100A0C00227540007541F022C2AF75C820A8CCA950
:100A1C00CDAA3A30CF010A75C824D2AFAB3BAC3C5F
:100A2C00883B893CC3E89BF8E99C206908F930664F
:100A3C00026125417FAD3D8A3DF9EA9DFA60067859
:100A4C00FF79FF4164AE3EAF3F8B3E8C3FA83BA984
:100A5C003CC3E89EF8E99FF9C3E54113FBE540135D
:100A6C00FAE82AF540E93BF54150067540FF75411F
:100A7C00FF41CCAA40AB41AC40AD417E047F02C3E8
:100A8C00EB9404400D1E1FC3EB94084005206A0232
:100A9C001E1FC3ED13FDEC13FCDEF7C3EA9CFAEB4F
:100AAC009DFBEF6009C3E913F9E813F8DFF7EA28B7
:100ABC00FAEB39FB8A408B4150067BFF8B408B4114
:100ACC00C3EB94025002D2663069047F0341F7787D
:100ADC0092E6FFC3E537948240110FC3E53794A02B
:100AEC0040010FC3EF940640027F057E02E541C42E
:100AFC00540FF9E541C454F0F8E540C4540F28F8FC
:100B0C00C3E89EFAE99400FB4009C3EA9402EB9413
:100B1C000050047A02E4FB6171AA40AB41EBC4FEC5
:100B2C00EAC4540F4EFCC3EA9CFAEB9400FBC3E8F6
:100B3C0013C313F8EA28FAEB3400FB8A408B41C349
:100B4C00EB94024002C2667802EBC4FE7B00EAC45E
:100B5C00540F4EFAC3EA98FA4005C3940250027A35
:100B6C00027892E6FF306002617185519285529352
:100B7C00D26043E680C3E49AF8E49BF930660261E4
:100B8C00FDE8FAE9FBD3E913FDE813FC885189521F
:100B9C00C3EF94036038EF20E00DE82CF8E93DF941
:100BAC00ECFAEDFB020BC6E828F8E939F9C3E824A6
:100BBC0002F8E93400F97AFE7BFFC3EF9403400E90
:100BCC008A538B54884D894E8C4F8D50813188536C
:100BDC0089548A4D8B4E8C4F8D503069127553F061
:100BEC007554FF754FF07550FF7551F07552FF81BC
:100BFC0031E8FAD3E813FC8851C3EF94036020EF7B
:100C0C0020E007E82CF8ECFA811DE8282402F87A99
:100C1C00FEC3EF940340088A53884D8C4F81318872
:100C2C00538A4D8C4FE568C3335002646BF56830C2
:100C3C006002813B753402D26043E680E52D540698
:100C4C006034A840A941C3E913F9E813F8C3E913C8
:100C5C00F9E813F8306904E92440F9C2AF53E67F90
:0F0C6C00759100C3E498F594E499F5957591049A
:100C7B00D26043E680D2AF22D26475430075200068
:100C8B00306C03752040020CA2D2647543007520B2
:100C9B0040306C0375200078017901206620E52D2A
:100CAB0054066002C2647914E541C313700104F861
:100CBB00C3941440027814306904781B791B2060AC
:100CCB0010E543600C306903D53404D26DA14C910F
:100CDB00430543E59B5440B52002A1363069090812
:100CEB00C3E89940011881C920640A08C3E89940F8
:100CFB000281A281C9C264C2AF53E67F75910030F5
:100D0B0066127594007595F8759104D26043E68070
:100D1B00D2AF81A2E5417EFFC3334005C33340010F
:100D2B00FEC3E49E759400F595A113C3E5339401BE
:100D3B00500281A230640281A2D802A14A81C9C2A9
:100D4B006DC2AF53E67F75910085539485549575AD
:100D5B009104854D92854E93D26043E680D2AFE5E8
:100D6B002D54066008206A020533020D88306D0D84
:100D7B00206C0A2064071581158102162C2278003D
:100D8B003064027801E53775F007A4F9E5F028F532
:100D9B00F0E9A2F013A2F113A2F213F537C3947882
:100DAB005003753778C3E53795384008D265C2953F
:100DBB00C294C293306002A1BF854F92855093D2EB
:100DCB006043E68022207D16C2AF754202D291C2EB
:100DDB0092306202D293D2AF759F11020FC0C2AF95
:100DEB00754202D291C290306202D295D2AF759FFA
:100DFB0011020FC0307243207D20C2AF75420390A9
:100E0B000135757B02C293D290306204D294C11D1E
:100E1B00C291D2AF759F01020FC0C2AF7542039052
:100E2B000135757B02C295D292306204D294C13DDA
:100E3B00C291D2AF759F21020FC0207D17C2AF7533
:100E4B004203900110C293306202D294D2AF759FCD
:100E5B0001020FC0C2AF754203900110C295306200
:100E6B0002D294D2AF759F21020FC0207D16C2AF64
:100E7B00754204D292C290306202D294D2AF759F67
:100E8B0021020FC0C2AF754204D290C292306202EF
:100E9B00D294D2AF759F01020FC0307243207D20D8
:100EAB00C2AF754205900124757B04C294D2913078
:100EBB006204D295C1C3C292D2AF759F11020FC00B
:100ECB00C2AF754205900146757B01C294D2913039
:100EDB006204D293C1E3C290D2AF759F11020FC0CF
:100EEB00207D17C2AF754205900106C29430620295
:100EFB00D295D2AF759F11020FC0C2AF754205904C
:100F0B00011AC2943062EBD293D2AF759F11020FCC
:100F1B00C0207D16C2AF754206D290C291306202DC
:100F2B00D295D2AF759F01020FC0C2AF754206D2E8
:100F3B0092C291306202D293D2AF759F21020FC041
:100F4B00307244207D20C2AF754201900146757B03
:100F5B0001C295D292306204D293E169C290D2AFB2
:100F6B00759F21020FC0C2AF754201900124757BA2
:100F7B0004C293D290306205D295020F8AC292D2EC
:100F8B00AF759F01020FC0207D17C2AF7542019054
:100F9B00011AC295306202D293D2AF759F21020F14
:100FAB00C0C2AF754201900106C293306202D29566
:100FBB00D2AF759F01C26522900104757B00C2956B
:100FCB00C294C293D292D291D290C262227880768E
:100FDB00070876070876010876040876FF0876FF7F
:100FEB0008760A087602087601087601788C760175
:100FFB000876000876B40876FF0876FF0876FF08B7
:10100B0076030876FF0876010876FF0876250876C2
:10101B00D00876780876C80876040876FF0876013B
:10102B0008760008767A08760A08760108760108B1
:10103B0076000876FF087600227887E6FFC2727882
:10104B0088C27DE630E102D27DC27E7889E630E14E
:10105B0002D27EC3EF94026008758E01D273021028
:0F106B0071758E00C273227880E6149000809316
:10107A0078A5F67881E6149000809378A6F67886AB
:10108A00E61490008D9378A7F6789FE6F8700575B8
:10109A006B0001B8C3E8941140027811E82828F5DA
:1010AA006B256B256B28F56C256B2828F56D7886E2
:1010BA00E6F539C394025003753902789CE675380F
:1010CA00FFB402037538A0B4030375388278A3E627
:1010DA001490009A93F566120FC322227896E6FAC4
:1010EA007897E6FB7888E6B40305C3EB940EFB30E9
:1010FA007F047A007BFFC3EB9AFCC3948250027C84
:10110A00827572000572EC8572F0A4C3E5F0947DD5
:10111A0040F222D27F11E61205561205567A007B5A
:10112A00007C1012054CE55C2AFA74003BFBDCF3E8
:10113A007C04C3EB13FBEA13FADCF7FEC27F11E669
:10114A0022757C00757D00E5EF20E6037520000519
:10115A0020903FFFE520146006901DFF1460009365
:10116A0004600375EF1653D9BF7581C043FF80121F
:10117A00054775EF0643B203E5B3240220E70DF5F0
:10118A0021E5E320E0068521B343E301120FC3758D
:10119A0080FF75A40075F19075D47F75908775A549
:1011AA00BF75F2BF75D50075A60175E241120FC36E
:1011BA00E4F8F6D8FD756801120FD81216837898EC
:1011CA008673753001C2AF1205601205701205569A
:1011DA0012057712055612057E1205561217B61217
:1011EA00056012056012055BC2AF757C00757D0053
:1011FA0078FA79FA308707D9FBD8F7021C0011442C
:10120A00117211E511E678988673120FC37588106A
:10121A0075890275C82475910475D84075A8227518
:10122A00B80275E690759B80759D0075D10E75BCE8
:10123A005875BB0675BA1175E880120547D2AF1208
:10124A00089F75360053DACF207E0343DA20307EBA
:10125A000343DA1043DA01C2D8C271120560D261BF
:10126A007B037A0CE55B70077A0CDB030211F2123E
:10127A0005562070030211F2C270E55CC394024065
:10128A00E1E52F541F855E5DF55EB55DD5DAD5C201
:10129A006153DACF207E0343DA20307E0343DA102B
:1012AA00C2D8C27178A2E67008D274E52F54E0F56C
:1012BA002FC27575290012055B307409C3E529949C
:1012CA000A4002D27512054C78023074027800C3C3
:1012DA00E55C9840F0C2AF120570120570120570F5
:1012EA00D2AF120560754C0012054C788CE6C39497
:1012FA000150030213DFE530C3940150030213DFE8
:10130A00757CA5757DF1207435C3E55C94FF5003A7
:10131A000213DFC2AF120585D2AF12055BC3E55CCB
:10132A00940150EFC2AF120570120551120570D226
:10133A00AF12055BC3E55C94FF40E902183B7F05E9
:10134A00D27F11E612055BC2AFC27F11E6AE5CC363
:10135A00E55C947FD2AF500261EF120547C2AF122B
:10136A000585D2AFDFDA311DC3EE94057897F61200
:10137A0005601217BE7F0AD27F11E612055BC2AF63
:10138A00C27F11E6AE5CC3E55C947FD2AF50E61231
:10139A000547C2AF120570120551120570D2AFDFB0
:1013AA00D6311DEE24037896F6F87997E7C394822E
:1013BA004003985006E824827897F61205601216C0
:1013CA00D11217ED12055B11E6C3E55C94FF5002DA
:1013DA00610A02183B757C00757D00C3E55C954C7B
:1013EA004003855C4C12055B78017988E7B40302F7
:1013FA007805C3E55C98400241F2C2AF1205851236
:10140A000585120585D2AF120560753000E4F53105
:10141A00F5320531E531F4703F0532789AE67819EC
:10142A00146012783214600D787D14600878FA140A
:10143A006003753200C3E53298401D120FC31205CE
:10144A0047153275310078998673C2AF120585D275
:10145A00AF7898867312055B120551E52A7005303C
:0F146A00740221F278012074027806C3E55C98C1
:1014790040A112055BE52A70030211F2C2AF120FF7
:10148900C3E4F522F523F524F525F526F567D2AF52
:101499007885E6C333F565E4F544F545F546F54742
:1014A900F548F570F52CF52DF53775700875BB10F5
:1014B90012054712093030EDFDA8BDA9BEE970013A
:1014C900F8887112093475700875BB101144C2AFE0
:1014D9007561FF1209ED852261852262852263D239
:1014E900AF7522017524017525017526018560698D
:1014F900756A017888E6B40307C27D307602D27D29
:10150900D268D269753300120F1C120F4B120A0DE3
:10151900120A14120A0D120A14120A0D120C94124C
:101529000666120D89120DD0120A14120C83306E40
:101539000312070620660312085930660312088948
:10154900120D89120DFF120A14120C94306E031237
:101559000742120D89120E76120A14120C83306E8C
:10156900031207A0120D89120EA5120A14120C9467
:10157900306E031207FD120D89120F1C120A141284
:101589000930120C83120D89120F4B120934120AF9
:101599001430692C856461856462856069756A01A6
:1015A90079187A0CC3E533994009C269D26A8A3538
:1015B9000215C9C3E55C94014003021525021634DE
:1015C900306A25206C22E535147006C26AD26BA1F7
:1015D90025F535C3E55C940140030215257888E6B5
:1015E900C394036003021634753600C3E55F9401A2
:1015F9004009856462856069756A0178FA79A4E7AA
:1016090060027803C3E55F985021307404E52A60CD
:101619001A78F0306C058564617820C3E5419850EB
:1016290002A1250536E55C6002C137753600C2AFF7
:10163900120FC37887E6FE760211447887EEF6E446
:10164900F522F523F524F525F526F565752C0075A4
:101659002D00D2AF12055B120FC378A4E66006C253
:1016690092C291C290307406E52A700221F2788DF7
:10167900E6C39401400241CF8117901A0D782012D8
:101689001713E520B4A50CA3121713E520B45A03C8
:101699000216B1757CA5757DF1120FD81216D17598
:1016A9007C00757D000216D0901A0378807B0A129F
:1016B9001713A308DBF9901A0F788C7B19121713EB
:1016C900A308DBF9901A2822C2AF12175612173352
:1016D900901A00740E121718A37409121718A3741C
:1016E90015121718901A0378807B0A121717A30886
:1016F900DBF9901A0F788C7B19121717A308DBF9FD
:10170900121769121747901A2822E493F622E64322
:101719008F01538FFDFFC3E583941C400122EF85A0
:101729007CB7857DB7F0538FFE22438F02438F012B
:10173900857CB7857DB7901A0DF0538FFC22901ADE
:101749000D74A5F118901A0E745AF118227A30798D
:10175900D07820901A40F113E520F709A3DAF7228F
:101769007A3079D0901A40E7F11809A3DAF922AB57
:1017790074A875BB01027980BB02027981BB03029F
:101789007982BB04027994BB05027983BB0602798D
:1017990086BB07027992BB08027987BB0902799C4B
:1017A900BB0A027988BB0B027989E8F7227C05120A
:1017B9000560DCFB22C2AF12057012057712057EA7
:1017C90012058512055112057012057712057E1250
:1017D900058512055112057012057712057E12054D
:1017E90085D2AF22C2AF12058512057E1205771286
:1017F900057012055112058512057E12057712052D
:101809007012055112058512057E120577120570B1
:10181900D2AF22AE74AF75C2AF1205701205701245
:101829000570120551DEF2120585120551DFF8D255
:10183900AF221217BE1217B61217B6757401757555
:1018490001757600111C7C05AD5C120560C3ED9530
:101859005C70F5C3E55C9401400AC3E55C94FF4004
:0F1869003702187E1217781216D11217BEC2AFAF
:1018780075EF161217B6DCD10576C3E576940350DA
:101888000280C21217B60575E5741490009F93F88C
:1018980008C3E57598500280A91217B61217B60545
:1018A80074C3E574940C50028095120FD81216D1A7
:0818B800C2AF75EF161217B65E
:0319FD0002114B89
:101A00000E091507070104FFFF0A020101A55A018B
:101A100000B4FFFFFF03FF01FF25D078C804FF01DA
:091A200000FF0A010100FF00FFB4
:101A400023585031384123202020202020202020DE
:101A500023424C48454C4923463333302320202031
:101A60002020202020202020202020202020202076
:101C0000C2AFC2D353D9BF7581C043B20343FF8073
:101C1000752438752503B1DC7529A5752AF175E29F
:101C20004043F18053A47F75D4FFD2877DFA7803B7
:101C300079E67C10752200752300901DE97B0675FE
:101C400024987525013087028145208708D8FBD963
:101C5000F9DCF781B7308708D8FBD9F9DCF781B711
:101C6000B19CE493A3C39A6004DDC381B7DBDBB10D
:101C70008E6002812E7B08E493FAA3B16FDBF87AC1
:101C800030B16F752200752300B18EEAFCEBFDC305
:101C9000ED94FE400EB18E8A278B28ED30E0048A49
:101CA000828B83B18E7AC270D8C3ED94FE601950D6
:101CB000CEBD002BEC600F7520007521FF7529004B
:101CC000752A000200008100A827A9280809D80465
:101CD000D90281DCB192EA89AAF281CE0D81A3C337
:101CE000ED94035053EDA2E092007AC5C3E58294CF
:101CF00000E583941C508A200010438F02438F011B
:101D00008529B7852AB7F0300029A827A92808090E
:101D1000438F01538FFDD804D902A133C3E58394C7
:101D20001C4003A3A11689AAE28529B7852AB7F02A
:101D3000A3A116538FFC817F7AC1BD030CE493A34A
:101D4000FAB153DCF8B14B817F8181AA22AB23B178
:101D50006FEBFAEA6222752608C3E52313F523E543
:101D60002213F52250066323A0632201D526EAB18F
:101D7000DCB1DC75260AEAF4200102D287300102C8
:101D8000C287B1DCC3134002C201D526EB22B19257
:101D9000EAFB208702A192308702A197752608AE40
:101DA00024AF25C3EF13FFEE13FEB1E0B1DCC3EAAD
:101DB000133087024480FA30E703632201C3E5232E
:101DC00013F523E52213F52250066323A0632201B5
:101DD000D526D9E52265236523F52222AE24AF2539
:101DE0000E0FDEFEDFFCD20122424C48656C6934E6
:071DF000373164F3300601F6
:00000001FF
